:100000000C947A040C94B2040C94B2040C94B204D0
:100010000C94B2040C94B2040C94B2040C94B20488
:100020000C94B2040C94B2040C948B140C94CD1365
:100030000C94441F0C94B2040C94B2040C94B204BB
:100040000C94B2040C94B2040C94B2040C94B20458
:100050000C941D220C9419160C94B2040C94B20446
:100060000C94B2040C94B2040C94B2040C94B20438
:100070000C94B2040C94B2040C94B2040C94B20428
:100080000C94B2040C94B2040C94B2040C94B20418
:100090000C94B2040C94B2040C94B2040C94B20408
:1000A0000C94B2040C94B2040C94B2041006120620
:1000B0006B061A0652062A067806DB064F07E30689
:1000C000AD06B106E706B406EA06F506BF06450723
:1000D000C306F906C706FD062707CB060107310749
:1000E000D10607071107B806EE06BB06F106D606CD
:1000F0000C071D073D073F07A906DF0658078107C4
:100100008707720778078D0793079907E50709089E
:100110000E08130818081D08220827082C083108A3
:1001200036083D0840084308460849084C084F086F
:10013000520855085A08BF08BF08F208F2087109AA
:100140008B0A8B0A8B0A8F09030A140A140A520EAF
:10015000550E910EBA0EC10ECC0ECF0ECF0ECF0E95
:10016000241024108A0F8C0F910FB70FD90FDC0FBA
:10017000DF0F0310E5110C12B5130C12B513581252
:100180007B12B51370138013B921AF21C721192237
:100190001B221B2219221B221B22E8211B22F221D7
:1001A000FC211B221B221B221B2219221B221B2289
:1001B00019221B22D5211B221B220C220C220C22CD
:1001C0000C220C220C220C220C220C2214221B22A8
:1001D000B921AC211B221B221B221B221B221B220A
:1001E0001B221B221B221B2214221B221B22192230
:1001F0001B220A220A220A220A220A220A220A228E
:100200000A220A2214220000000000000000000060
:1002100000000000000000000000000000000000DE
:10022000000000000000000000007E0F00D4FFFF6F
:10023000FFC70000007800000000000000002A2B2B
:100240002800000000000000000000000000000086
:100250000029000000002C1E3420212224342627EF
:10026000252E362D3738271E1F2021222324252610
:100270003333362E37381F0405060708090A0B0CDE
:100280000D0E0F101112131415161718191A1B1C26
:100290001D2F3130232D350405060708090A0B0CE4
:1002A0000D0E0F101112131415161718191A1B1C06
:1002B0001D2F3130354C1E0F0500047F3F1F643267
:1002C00014643214783C1E1E140A0505010980A12D
:1002D00001850319012AB700150126B7009501759C
:1002E000108100C0050C0901A101850419012AA093
:1002F00002150126A002950175108100C0050109B3
:1003000006A1018506050719E029E71500250195D5
:1003100008750181020507190029EF1500250195CF
:10032000F0750181020508190129059505750191EE
:1003300002950175039101C00660FF0961A10109E1
:1003400062150026FF0095207508810209631500DB
:1003500026FF00952075089102C005010906A1013C
:10036000050719E029E715002501950875018102A7
:100370009501750881010507190029FF150026FF61
:100380000095067508810005081901290515002545
:1003900001950575019102950175039101C009024E
:1003A0005B00030100A0FA09040000010301010041
:1003B0000921110100012244000705810308000101
:1003C00009040100020300000009211101000122BB
:1003D0002200070582032000010705030320000116
:1003E000090402000103000000092111010001229B
:1003F0006D000705840320000112010002000000C7
:1004000008756F7368010001020001120331007565
:100410000070003600300068007300650000001AAC
:10042000033100750070006B006500790062006F99
:1004300000610072006400730000000403090422DC
:1004400023252628292A2C2D2F3032333536383AC9
:100450003B3D3E4042434547494A4C4E505153551F
:1004600057595A5C5E6062646668696B6D6F717340
:100470007577797B7D7F81838587898A8C8E909241
:100480009496989A9C9E9FA1A3A5A7A8AAACAEAF4C
:10049000B1B3B4B6B8B9BBBCBEBFC1C2C3C5C6C791
:1004A000C9CACBCCCDCED0D1D2D2D3D4D5D6D7D742
:1004B000D8D9D9DADADBDBDBDCDCDCDCDCDDDDDD8A
:1004C000DDDCDCDCDCDCDBDBDBDADAD9D9D8D7D786
:1004D000D6D5D4D3D2D2D1D0CECDCCCBCAC9C7C633
:1004E000C5C3C2C1BFBEBCBBB9B8B6B4B3B1AFAE71
:1004F000ACAAA8A7A5A3A19F9E9C9A989694929017
:100500008E8C8A89878583817F7D7B7977757371EE
:100510006F6D6B6968666462605E5C5A59575553CB
:1005200051504E4C4A4947454342403E3D3B3A3884
:1005300036353332302F2D2C2A2928262523220028
:10054000000000000000000000000101020304059B
:1005500006080A0C0F1114181C2024292E33393FC9
:10056000464C535B626A7179818A929AA2AAB2B9A7
:10057000C1C8CFD5DCE1E7EBF0F4F7FAFCFDFEFFF4
:10058000FEFDFCFAF7F4F0EBE7E1DCD5CFC8C1B92A
:10059000B2AAA29A928A8179716A625B534C463FF1
:1005A00039332E2924201C1814110F0C0A080605B3
:1005B0000403020101000000000000000000002907
:1005C000001E001F0020002100220023002400251F
:1005D00000260027002D002E002A002B0014001AF0
:1005E000000800150017001C0018000C0012001372
:1005F000002F003000310039000400160007000908
:10060000000A000B000D000E000F00330034000044
:10061000002800E1001D001B000600190005001164
:1006200000100036003700380000000000E500E050
:1006300000E300E200000000002C000000000000C9
:1006400000E600E70021520000E40035003A003BDC
:10065000003C003D003E003F00400041004200439E
:1006600000440045004C000100010052000100015F
:1006700000010001000100010001004600470048A0
:100680000001000100500051004F00010001000175
:10069000000100010049004A004B00000001000178
:1006A00000A900AA00A8000100010001000100014A
:1006B000004D004E0000000000010001000100019B
:1006C0000000000000010000000000000001002206
:1006D00052010000000100010001000100010001C1
:1006E0000001000100010001000100010001000102
:1006F00000007C027804780378057801000100018D
:1007000000010001000100010001000100010020C2
:1007100078217823782578277829782B782C782DDC
:10072000782E7801000100000001000100227824E9
:1007300078267828782A782F7830783178327801BE
:1007400000000000000100010001000100000000A5
:100750000001000000000000000100010001000095
:100760000001000100010001000100010001000181
:100770000001000100010001000100010001000171
:100780000001000100010001000100010001000161
:100790000001000100010001000100010001000151
:1007A0000001000100010001000100010001000141
:1007B0000001000000010001000100010001000132
:1007C0000001000100010001000100010000000023
:1007D0000001000100010001000000000001000014
:1007E0000000000000010001000100000001000005
:1007F00001010101010101010102020202020202E2
:1008000002020303030303030303040404040404B4
:10081000040505050505060606060607070707077A
:1008200008080808090909090A0A0A0B0B0B0C0C2D
:100830000C0D0D0D0E0E0E0F0F0F101011111112C9
:100840001213131414151516161717181819191A48
:100850001A1B1B1C1D1D1E1E1F20202122222324AB
:1008600024252626272829292A2B2C2D2D2E2F30EA
:10087000313232333435363738393A3B3C3D3E3FFE
:10088000404142434445464748494A4C4D4E4F50EB
:10089000515354555658595A5B5D5E5F61626465A9
:1008A0006668696B6C6D6F7072737577787A7B7D33
:1008B0007E8082838587888A8C8E8F919395969887
:1008C0009A9C9EA0A2A3A5A7A9ABADAFB1B3B5B7A3
:1008D000BABCBEC0C2C4C6C9CBCDCFD1D4D6D8DB7A
:1008E000DDDFE2E4E7E9EBEEF0F3F5F8FAFDFFFF18
:1008F000AA7F554011241FBECFEFDAE0DEBFCDBF87
:1009000004B603FE18C08091310390913203A09188
:100910003303B09134038730904BA740B04B59F468
:100920001092310310923203109233031092340369
:10093000E0E0F8E3099511E0A0E0B1E0ECE8F7E5CC
:1009400002C005900D92A43AB107D9F723E0A4EABA
:10095000B1E001C01D92A133B207E1F70E94130B71
:100960000C94C42B0C940000A8E0B0E0EAEBF4E097
:100970000C943C2BFC018481882309F450C67F0130
:1009800021E0408151816281738195810E94EC2830
:100990008C01F7018581882309F4B4C19801375788
:1009A0002038310508F032C1003108F0DBC28FEF8A
:1009B00093E00E94132A8111D5C238E5A32E32E0BC
:1009C000B32E002379F0A114F4E0BF0609F4CAC2E3
:1009D000C5010E94132A811101C001502FEFA21AF4
:1009E000B20AEFCFCE0101962C0188E0F2011192FC
:1009F0008A95E9F72AE0322E85010F5F1F4FC50166
:100A00000E94132A89831A82882309F4ABC2813099
:100A100009F041C06501F2E0CF0ED11CC8010E946F
:100A2000132A8A83882309F49DC29FEF980F93307D
:100A300060F423E0A20EB11CC6010E94132A8B832E
:100A4000882309F48FC21C8229C0843031F54E01FD
:100A500033E0830E911C02E010E056018FEFA81ADC
:100A6000B80AC6010E94132AF40181934F0188231A
:100A700009F478C28C3741F4E2E0F0E0EC0FFD1F9E
:100A8000E00FF11F10820AC00F5F1F4F6501073092
:100A9000110519F767C2580101C056018201F8011A
:100AA0002081222309F4A8CF213009F053C081818D
:100AB000813081F46801F2E0CF0ED11CF80182810F
:100AC000893319F460E570E002C060E070E00E94D4
:100AD000131B15C0823049F46801F2E0CF0ED11C1F
:100AE000F80182810E94361A0AC0833051F46801ED
:100AF000F2E0CF0ED11CF80182810E94E519860137
:100B000082C0843019F00F5F1F4F7DC0F801228131
:100B10000E5F1F4F80E090E030E0205331092A3013
:100B2000310568F4389EA001399E500D1124C90189
:100B3000840F951F0F5F1F4FF8012081EDCF0097A5
:100B400009F461C0EFE9FFE03197F1F700C0000060
:100B50000197F5CFE22FF0E0EA5CFD4F2490822F61
:100B600086958695869590E0FC01EA5DFD4F649040
:100B70002770712C022E02C0759467940A94E2F7D4
:100B8000F1E06F227724FC01EA5EFD4F8490912C06
:100B9000022E02C0959487940A94E2F731E08322F2
:100BA0009924FC01EA5FFD4FC490D12C02C0D5947A
:100BB000C7942A95E2F781E0C822DD24611471040C
:100BC00019F081EE0E94361A8114910419F086EE14
:100BD0000E94361A60E070E0822D0E94131B81147F
:100BE000910419F086EE0E94E5196114710419F060
:100BF00081EE0E94E519C114D10429F060E070E093
:100C00008CE20E94131B0F5F1F4F49CFF801F8576A
:100C1000E730F10508F076C0EA5AFF4F0C94202B1C
:100C200085E001C080E00E94391C8091F0020E94A2
:100C3000081C98C18091F002982F969596959695EC
:100C400049F1915E990F990F990F8770892B8093C5
:100C5000F00214C09091F002892F869586958695B2
:100C60008F5F8F719770863008F03FC0880F880FB4
:100C7000880F892B8093F0028091F002887F91E0A9
:100C800009F490E08091F00290FB80F98093F002EB
:100C90000E94081C8091F0028695869586950E9498
:100CA000962260C12091F002822F869586958695C6
:100CB000482F50E04530510554F48F5F982F990F1D
:100CC000990F990F822F8770892B8093F002809162
:100CD000F0028160DBCF8091F00280FF03C00E94B0
:100CE000531C40C10E94601C3DC19093F002C4CFD0
:100CF0008091F00281FF03C00E940E1C33C10E944C
:100D0000241C30C1F801E851FC47E730F10508F434
:100D1000E5C0882309F446C11092F802C801905733
:100D2000839708F00CC184E090E00E94212A909300
:100D300000038093FF02F801E150F047E232F10531
:100D400020F4E35AFF4F0C94202B8091FF02816026
:100D5000ACC0809100038860B4C08091FF028260C3
:100D6000A4C08091FF0220C08091FF0288609DC0D6
:100D7000809100031EC0809100038260A2C0809118
:100D8000FF02806192C08091FF0280628EC08091DC
:100D9000FF0280648AC00E94B2198091FF028068BD
:100DA00084C08091FF02886084607FC080910003CE
:100DB0008260816086C08091FF028E7F76C08091C4
:100DC0000003877F7EC08091FF028D7F6EC080917F
:100DD000FF0220C08091FF02877F67C080910003DF
:100DE0001EC0809100038D7F6CC08091FF028F7EBA
:100DF0005CC08091FF028F7D58C08091FF028F7B85
:100E000054C00E94B2198091FF028F774EC080912A
:100E1000FF02877F8B7F49C0809100038D7F8E7F8B
:100E200050C08091FF0282FB222720F991E0922797
:100E300090FB82F990FB83F938C080910003982FD2
:100E4000909591708E7F892B90FB81F93AC08091AB
:100E5000FF0286FB222720F991E0922790FB86F97A
:100E600024C00E94B2198091FF0287FB222720F93B
:100E700091E0922790FB87F918C061E001C060E023
:100E80008EE090E00E94372A1EC08091FF0284FB12
:100E9000222720F991E0922790FB84F906C08091E7
:100EA000FF02982F909590FB80F98093FF020BC072
:100EB0008091000383FB222720F991E0922790FB89
:100EC00083F9809300036091FF027091000384E036
:100ED00090E00E94552A0E94B21944C0E158FF4F89
:100EE0000C94202B06E221EE41EE6AE17CE705C07E
:100EF00007E225EE45EE6BE17CE7C7010E94662024
:100F000031C006E221EE40EE68E17CE7F6CF07E271
:100F100025EE44EE69E17CE7F0CF06E221EE42EEF9
:100F20006CE17CE7EACF07E225EE46EE6DE17CE777
:100F3000E4CF08E221E045EE6EE17CE7DECF06314A
:100F4000FCE71F0719F580912A038A7A91E009F4DA
:100F500090E09093A601811117C089E20E949B1F27
:100F60000E94492680914202877009F458C3F70114
:100F70008581882309F453C38091000382FF4FC306
:100F800082E00E9475194BC385E3E8CF07372CE751
:100F9000120709F4F2C208373CE7130709F0FDC253
:100FA00082E0EFC206318CE7180709F4DCC28091B9
:100FB0002A038272F801E052F847E531F10508F0A2
:100FC0007EC0EA57FF4F0C94202B8091C00280FF17
:100FD00019C0282F2E7F2093C0023091C10240916A
:100FE000C2025091C3026091C4027091C502809107
:100FF000C6029091C7020E94C02610924C020E9425
:10100000D21CB0CF81608093C00261E08695869546
:101010004EC045ED58E260EE78E22CC040EE58E25A
:1010200065ED78E227C041E758E26BE778E222C03D
:101030004BE758E261E778E21DC047E558E264E615
:1010400078E218C044E658E267E578E213C04DE361
:1010500058E26AE478E20EC04AE458E26DE378E2CE
:1010600009C046EE56E260E077E204C040E057E295
:1010700066EE76E20E94B41C75CF61E081E017C095
:1010800065E082E019C068E086E016C06EE089E0A5
:1010900013C064E18FE010C067E185E10DC061E03D
:1010A00088E105C062E289E107C061E083E20E9455
:1010B000852858CF6AE285E20E949F1C53CF0737EC
:1010C000FCE71F0709F45BC208372CE7120709F495
:1010D0005BC2F701858100811181882349F0C80135
:1010E0000E94F416D82E682FC8010E940E1904C061
:1010F000C8010E94DA18D82EB8018D2D0E948624CE
:101100000E949424D82E192FA82EF7010581C6809D
:10111000C2949FE0C92280914202877001F10023AE
:10112000F1F0812F807F803469F080E28D0D88306E
:10113000B0F0812F807E803229F4F1E0FD1578F443
:10114000CC2069F08091000382FF09C082E00E94F8
:101150007519809142028770BB24B3948111B12C20
:10116000912E92948FE09822892D90E08C309105F9
:1011700008F0D1C1FC01E556FF4F0C94202B812FC4
:10118000807F1F70882311F01295107F0023B9F023
:10119000112309F4AEC180E28D0D883010F0A1104A
:1011A00006C090912A03192B10932A0305C0909131
:1011B0004402192B109344020E9449269AC18D2D96
:1011C0000E94E519112309F4A6C180E28D0D883033
:1011D00088F1AA2079F11095909144021923109377
:1011E00044022BC0812F807F1F70803211F0129536
:1011F000107F8D2DAA2029F021E0A21609F44CC001
:1012000057C08091000382FD1BC0002369F01123A9
:1012100039F090912A03192B10932A030E94492632
:1012200080E00E94361A77C180E00E94E519112300
:1012300009F471C1812F0E9442260E9449266BC188
:10124000002381F0CC20C1F131E0C31264C1909140
:101250004302812F8923181709F45DC1192B1093BC
:10126000430259C1C11057C1812F0E94D4198091E6
:101270004302912F982329F0912F909589238093F1
:1012800043022091A701812F822309F444C11095C4
:1012900021232093A7013FC1002329F085E08C156D
:1012A00008F439C109C094E09C1508F434C115C094
:1012B000002331F0C1101DC1812F0E94DB192BC109
:1012C000CC2059F0893309F023C1EFEFF7EE23E08A
:1012D000E150F0402040E1F719C1812F0E94D4195C
:1012E0001AC1812F86958695837019F0813061F03F
:1012F00012C1002321F08D2D912F937002C080E048
:1013000090E00E94F71F0DC1002321F08D2D912F39
:10131000937002C080E090E00E94D21F02C1812F32
:101320008370A9F50111FBC04D2D4295469547707C
:10133000440F440F8D2D8F7090E09C01042E01C04E
:10134000220F0A94EAF7D4FE08C08FE090E001C0B3
:10135000880F4A95EAF7809501C080E016951695AA
:101360001370123069F088F490912B03113019F04A
:10137000822B892302C0922B892B0E94AF19CFC0E8
:10138000822B90912B038927F8CF822BF6CF002355
:1013900019F0812F817001C08695882309F4BFC0A0
:1013A0004D2D429546954770440F440F8D2D8F70FB
:1013B00090E09C01042E01C0220F0A94EAF7D4FEAB
:1013C00008C08FE090E001C0880F4A95EAF7809549
:1013D00001C080E0169516951370123059F078F41C
:1013E0009091B201113019F0822B892309C0922B00
:1013F000892B06C0822B9091B201892701C0822BD4
:101400000E9443198CC01F70002339F0812F0E9465
:10141000A3198D2D0E94DB1982C08D2D0E94D41935
:10142000812F0E9468197BC08D2D32EFA31681F1A8
:101430003A1538F090EFA91659F0E1EFAE1619F110
:1014400054C0F3EFAF1659F124EFA216C1F04DC00E
:10145000002381F034E03C1508F45DC01F7181E089
:1014600090E0012E01C0880F0A94EAF79091B20132
:10147000892720C085E08C1508F44DC0EFCF8091FE
:10148000000382FD1AC0002329F0812F8F7120C034
:101490000023D9F3812F8F710E9468193CC000236B
:1014A00041F01F7181E0012E01C0880F0A94EAF714
:1014B00001C080E00E9443192EC0002361F0812FFB
:1014C0008F7198E0899F900111242360209342023C
:1014D0000E94A31920C081E00E947519E1E0EC157B
:1014E000D0F482E00E94751916C0002321F0CC20B0
:1014F00061F28D2D96CECC2069F2893349F4FFEF4D
:1015000027EE33E0F15020403040E1F700C000000A
:101510008D2D0E94E51988EF890D843010F40E940A
:101520001C20BB20A9F08091420280FD11C0F70170
:1015300015828695869586950E94A319C7010E94FB
:10154000B404809142028695869586950E9468191A
:1015500020E0F7014081518162817381848195810E
:101560000E94EC285CC08091A601811104C089E230
:101570000E946D1FF5CC85E3FBCF81E002C081E0C6
:1015800004C00E94A31903C082E00E94681943E0CE
:1015900062E081E00E944619E5CC03309CE7190720
:1015A00049F46FEF7FEF80E090E00E94552A0E949F
:1015B000A129D8CC0430ECE71E07B8F40115FCE7EC
:1015C0001F0771F40E94B2199FEFE4E3FCE0915011
:1015D000E040F040E1F700C000000E94F515C2CCE9
:1015E00001302CE7120719F374CD0B353CE71307D4
:1015F00021F480E00E948C196CCD0C358CE7180723
:1016000041F48091000382FB882780F991E08927CB
:10161000F1CF0A351C4709F05CCD81E0EBCF28966D
:10162000E2E10C94582BA6E2B0E0E9E1FBE00C9477
:101630003C2B85B7806885BF85B7806885BF84B738
:10164000877F84BF0FB6F894A89580916000886169
:1016500080936000109260000FBE90E080E80FB6AB
:10166000F89480936100909361000FBE81EC92E248
:101670009093A5018093A4010E9411140E9430143C
:101680008091E20084608093E20078948091DC0194
:101690008823A1F01091E9001F709091EC00892F30
:1016A000817090FD80E8182B1092E9008091E8008D
:1016B00083FD0E9402111F701093E90082E084BD37
:1016C00093E095BD9AEF97BD80936E000E944D20E8
:1016D000811102C00E9462210EE111E043E2E42E7A
:1016E00041E0F42ED8018D918D018F3F11F00E94C1
:1016F000AE23E016F106B1F703E211E031E3E32E89
:1017000031E0F32EF80181918F018F3F11F00E949B
:10171000AE23E016F106B1F78AE0E1ECF1E0DF017B
:10172000282F1D922A95E9F7E8EAF1E0DF011D92E2
:101730008A95E9F780E090E00E94212A853E9E4F3D
:1017400021F40E944D20811102C00E94D52582E023
:1017500090E00E94132A8093F50284E090E00E94BA
:10176000212A909300038093FF020E94C523EFEF8C
:10177000F6E721E0E150F0402040E1F700C0000032
:101780000E94C5238091C10180FF08C06FEF7FEFE9
:1017900080E090E00E94552A0E94F51583E090E0D9
:1017A0000E94132A0E94AF19279A2F988AE08093EB
:1017B000800089E1809381008FEF9FEF90938700F5
:1017C000809386000E94781C8091F00281FF0BC0FC
:1017D0001092F3021092F2021092F10280916F00C7
:1017E000816080936F000E94781C8091B301811109
:1017F0007FC088E090E00E941B2A4B015C0183E2DD
:1018000090E00E94132A282F30E040E050E060E092
:1018100070E080E090E000E20E94732B28293929D3
:101820004A295B292093C0023093C1024093C2022F
:101830005093C3026093C4027093C5028093C602A2
:101840009093C7022C7F09F041C025E02093C0028D
:101850001092C1023FEF3093C2023093C302109244
:10186000C40230E04FEF5FEF60E00E94C02688E0E6
:1018700090E00E941B2A6B017C0183E290E00E94B1
:10188000132A282F30E040E050E060E070E080E074
:1018900090E00E94732BB22FA32FF42FE52F5B0152
:1018A00097018601BC29A12BF22BE32BB093C00238
:1018B000A093C102F093C202E093C3026093C402FA
:1018C000B092C5028093C6029093C7020E94AC26D4
:1018D00010924C020E940C1F8091C00280FF05C034
:1018E00060E0869586950E94852881E08093B3010B
:1018F00084E091E09093FC028093FB0228E1422E69
:10190000512C8E010F5F1F4F8091DC01853009F053
:1019100069C080E1E82E92E1F92E8091DC018530EA
:1019200009F051C08091DC01843009F439C080E0B5
:101930000E94391C10924C028091B50181110EC099
:1019400081E08093B5018091C002982F91709093AF
:10195000B4018E7F8093C0020E94D21C10920103BA
:1019600090E40FB6F894A895409260000FBE909353
:10197000600083B7817F846083BF83B7816083BF4A
:101980007894889583B78E7F83BF0FB6F894A89517
:1019900080916000886180936000109260000FBEAB
:1019A0008091DB01882309F4B8CF0E94C523E1ECC4
:1019B000F1E081919191892B09F04FC3A1E0EB3CBB
:1019C000FA07B9F7AACF0E94B2190E94781C0E94A8
:1019D0001C201092B5018091B40181110E94CA2887
:1019E0000E94BB1C0E94C523A6EBEA2EA1E0FA2EA2
:1019F000B1EC6B2EB1E07B2ED301F7012191319137
:101A00008D919D918227932721E0E03CF20719F008
:101A1000892BA1F305C0892B19F40E94B1253FC081
:101A2000312CD3018D909D903D01F701A080B180B4
:101A3000A824B924A114B10449F1212CCC24C394C5
:101A4000D12CC5018C219D21892BB9F029A23AA264
:101A50000E94381F9CA38BA3F1E0FDA391E09401A9
:101A60002C213D21232B09F490E09EA349A15AA1EA
:101A70006BA17CA18DA10E9411292394CC0CDD1CAB
:101A80002EE02212DECFD7018D929C923394B2E0E9
:101A9000EB0EF11CE5E03E12C4CF0E943F16809190
:101AA0004C02882309F4ABC080914B02E091C00244
:101AB000E695E695E81BE0934702823059F4F0E0A2
:101AC000E953FD4FE491EE2EF12C76E7C72E7BE132
:101AD000D72E70C0863059F4F0E0EC53FD4FE491FE
:101AE000EE2EF12C66E6C62E6BE1D62E63C0893051
:101AF00061F4E695F0E0EF53FD4FE491EE2EF12C0A
:101B000052EEC52E5EE1D52E55C08F3061F4E695BC
:101B1000F0E0E254FD4FE491EE2EF12C4DE7C42E9F
:101B20004EE1D42E47C0853159F4F0E0E554FD4F25
:101B3000E491EE2EF12C3FE2C32E3EE1D32E3AC0CB
:101B40008831F9F0833249F4E9EBF2E0E590F49062
:101B50002CE2C22E2BE1D22E2DC08432D1F0853260
:101B600009F58E2F63E00E94DE2AE92FF0E0EA54A7
:101B7000FD4FE491EE2EF12C98EEC92E9CE1D92E6A
:101B800019C0B8E2EB2EF12C84EBC82E8DE1D82ED3
:101B900011C0F4EFEF2EFF24F394ACE7CA2EADE1B1
:101BA000DA2E08C070EDE72E77E0F72EEBE2CE2EAE
:101BB000EBE1DE2E80914802882361F0109248020A
:101BC0000E94381F909346028093450210924A0269
:101BD000109249020E94381FE0914502F09146029E
:101BE0008E1B9F0B8F3F9F4750F4EE0EFF1EF0920F
:101BF0004602E092450285E492E0F60109950E94D2
:101C00001C209091C001891721F08093C0010E948F
:101C10003F168091DC01843009F076CE83E080931A
:101C2000E9008091E80082FF6FCE8091E80085FF97
:101C300023C00E94621581111DC060E2E62EF12CC6
:101C4000CE0101966C0109C08091F100D6018D93FF
:101C50006D01B1E0EB1AF10869F08091E80085FDB3
:101C6000F3CF8091E8008B778093E8000E946215A3
:101C7000882399F391E001C090E08091E8008B7790
:101C80008093E800992309F43FCE2981822F90E0C8
:101C9000FC013197E331F10508F0D6C1E955FF4F5A
:101CA0000C94202B1A828CE03AC18A81823009F48C
:101CB000EAC150F4813009F0C7C10E943F169B83EE
:101CC0008C837D836E83C2C1833041F0843009F000
:101CD000BBC11B821C821D821E82B8C14B81DE01EA
:101CE000119680E090E0242F30E0B901680F791F51
:101CF0006530710508F0AAC1E42FE80FF0E0EE0F9F
:101D0000FF1FEF53FE4F5081618113966C93139721
:101D100014965C931497019612968E30910529F7CC
:101D200095C18A81823019F0853051F08DC16B8167
:101D30007C818D819E810E94262B0E94292086C154
:101D40008091F00280FF03C00E94531C02C00E94D9
:101D5000601C8091C00280FF0AC08091C0028E7F0B
:101D60008093C00210924C020E94D21C6FC10E944C
:101D7000CA286CC14C816B818A810E9472219D832B
:101D800089C12D813E813227232732274C816B81E7
:101D90008A810E9406215AC10E942D2157C18A8141
:101DA0008130E1F52830F1F0293099F18B818130D3
:101DB00019F0823071F04AC18C81E5E08E9FC0013C
:101DC00011246FEF70E00E94F82A862F0E94391CC0
:101DD0003DC18C81811103C00E940E1C37C10E943D
:101DE000241C34C18B81813041F0823009F02EC136
:101DF0008091F0028695817078C08091F00286957E
:101E000086958695FFEF8F9FC001112465E070E0F5
:101E10005DC08091F0020E94081C18C1823009F058
:101E200013C12830B9F1293009F461C08B818230A7
:101E3000F9F098F4813009F009C18C812FEF829F6D
:101E4000C00111246FEF70E00E94F82A462F20E0B5
:101E50006091C2028091C1021AC08330A1F0843027
:101E600009F0F4C020E04091C3026D818C810FC065
:101E70008C81882309F471CF0E94CA2860E08C818C
:101E80000E948528E3C08C818093C402DFC00E9439
:101E9000BE27DCC08B818230E9F060F4813009F02C
:101EA000D5C08091C302AFEF8A9FC00111246FEFAC
:101EB00070E00CC08330B9F0843009F0C7C0809165
:101EC000C1028C838091C2028D83C0C00E94F82A17
:101ED0006C83BCC08091C00280FF03C0869586954C
:101EE00004C080E002C08091C4028C83AFC0209106
:101EF000C0023091C1024091C2025091C302609170
:101F0000C4027091C5028091C6029091C7020E94DE
:101F1000C0269CC080E151C0B1E0BA8388EA8B83BF
:101F200095C0EA80FB80FE24EF24FE24CC80D12CD7
:101F30005801C701885A9D4F9501201B310B2C1564
:101F40003D0508F083C0E8EAEE16E1E0FE0630F455
:101F50000E94132AD50114968C9302C0F5011482B5
:101F6000FFEFEF1AFF0A2FEFA21AB20AE2CFEA80C0
:101F7000FB80FE24EF24FE24CC80D12C5801C70125
:101F8000885A9D4F9501201B310B2C153D0508F0FB
:101F90005DC0A8EAEA16A1E0FA0620F4F501648122
:101FA0000E94372AFFEFEF1AFF0A2FEFA21AB20A98
:101FB000E6CF0E94F6204AC084E08A8347C0EA80C8
:101FC000FB80FE24EF24FE24CC80D12C5801C701D5
:101FD00088969501201B310B2C153D05B8F5A0E323
:101FE000EA16A2E0FA0628F40E94132AF501848377
:101FF00003C0D50114961C92BFEFEB1AFB0AEFEF5A
:10200000AE1ABE0AE4CFEA80FB80FE24EF24FE2451
:10201000CC80D12C5801C70188969501201B310B2B
:102020002C153D0598F4F0E3EF16F2E0FF0628F4D6
:10203000D50114966C910E94372ABFEFEB1AFB0A68
:10204000EFEFAE1ABE0AE7CF8FEF898340E250E090
:10205000B80182E00E94951557CCE9BCF9BC09B4DF
:1020600000FEFDCF8091D8008F7D8093D8008091B5
:10207000E00082608093E0008091E00081FDFCCF71
:102080000E94B2194ACC87E290E00E94132A1B8278
:102090001C821D828E83DACF8091DE0187FF11C002
:1020A0008091E80082FD05C08091DC018111F8CFAC
:1020B00011C08091E8008B770BC08091DC018823F0
:1020C00049F08091E80080FFF8CF8091E8008E779A
:1020D0008093E8000895982F973068F59093E90071
:1020E000981739F07091EC002091ED005091F000BC
:1020F00003C0242F762F50E021FD02C09F5FECCF5C
:102100003091EB003E7F3093EB003091ED003D7F4E
:102110003093ED003091EB0031603093EB00709321
:10212000EC002093ED005093F0002091EE0027FD8D
:10213000E5CF80E008958F708093E90081E00895F5
:102140002091E4013091E5012617370748F0611529
:10215000710539F42091E8002E772093E80001C042
:10216000B901FC0120E06115710579F18091DC0174
:102170008823F1F18530F1F18091E80083FD3CC0C6
:102180008091E80082FD2EC08091E80080FFEBCFB7
:102190002091F3008091F20090E0922B611571057F
:1021A00051F08830910538F421912093F10061506D
:1021B00071090196F3CF21E0089709F020E08091A2
:1021C000E8008E778093E800CECF2111CFCF0AC0F0
:1021D0008091DC01882361F0853061F08091E80016
:1021E00083FD0AC08091E80082FFF2CF80E008956D
:1021F00082E0089583E0089581E008950895809134
:10220000D1010895AAE2B0E0E8E0F1E10C944B2B93
:10221000EEEDF1E086EE91E02091F10021938E1732
:102220009F07D1F78091DF01833009F463C030F458
:10223000813071F0823009F49DC0B4C08A3009F455
:1022400089C08B3009F46EC0893009F0ABC020C062
:102250008091DE01813A09F0A5C08091E800877F76
:102260008093E8008091E2019091E301892B21F4B1
:1022700068E082ED91E003C060E080E090E070E013
:102280000E94A0108091E8008B778093E8008AC0BC
:102290008091DE01813209F085C08091E201909148
:1022A000E301009719F0029709F07CC08091E800E3
:1022B000877F8093E8008091E80082FD05C08091CF
:1022C000DC018111F8CF6EC02091F3008091F20003
:1022D00090E0922B029731F48091F100813011F05F
:1022E000863021F48091F1008093D1018091E80043
:1022F0008B7754C08091DE01813A09F053C0809100
:10230000E2019091E301892B09F04CC08091E80033
:10231000877F8093E8008091E80080FFFCCF809168
:102320000E0137C08091DE018132E1F58091E2013A
:102330009091E301892BB1F58091E800877F80932C
:10234000E8000E944C108091E00180930E010E94F1
:10235000B21928C08091DE01813221F58091E80018
:10236000877F8093E8000E944C108091E101809368
:10237000D00118C08091DE01813AA1F48091E8007B
:10238000877F8093E8008091E80080FFFCCF8091F8
:10239000D0018093F1008091E8008E778093E8006F
:1023A0000E944C108091E80083FFDFC18091DE0124
:1023B0009091DF01492F50E04A30510508F0D5C116
:1023C000FA01E654FF4F0C94202B803821F082381C
:1023D00009F0CBC108C08091DA019091DB0199230B
:1023E00089F082600FC08091E2018F70873008F021
:1023F000BCC18093E9008091EB0085FB882780F9C0
:102400001092E9009091E800977F9093E800809304
:10241000F1001092F10070C1282F2D7F09F0A5C1A5
:10242000882319F0823061F0A0C18091E0018130F1
:1024300009F09BC1933009F080E08093DB012EC04E
:102440008091E00181112AC08091E2018F702FEF0D
:10245000280F263008F089C18093E9002091EB0015
:1024600020FF1CC0933021F48091EB00806214C0E7
:102470009091EB0090619093EB0021E030E0A90196
:1024800002C0440F551F8A95E2F74093EA0010926C
:10249000EA008091EB0088608093EB001092E900E5
:1024A0008091E800877F8093E8000E944C105DC116
:1024B00081115BC11091E0011F778091E30080786A
:1024C000812B8093E3008091E800877F8093E80070
:1024D0000E944C108091E80080FFFCCF8091E300C7
:1024E00080688093E300111102C082E001C083E0A4
:1024F0008093DC013AC18058823008F036C12091C7
:10250000E0013091E1012C3D53E0350779F583E09E
:102510008A838AE289834FB7F894DE01139620E01C
:102520003EE051E2E32FF0E050935700E49120FFAA
:1025300003C0E295EF703F5FEF708E2F90E0EA30BE
:1025400010F0C79601C0C0968D939D932F5F2431E4
:1025500049F74FBF8091E800877F8093E8006AE2E7
:1025600070E0CE0101960E94A010B4C08091E201FB
:102570009091E301432F552743305105A9F068F4AA
:102580004130510509F400C14230510509F0EDC058
:102590008BE590E0EEE9F3E04BC04132510529F1C3
:1025A0004232510589F1E1C0C90199278130910575
:1025B000A1F058F0029709F0D8C0EBE0F4E0E49104
:1025C0008E2F90E0EBE0F4E030C0EBE3F4E0E49138
:1025D0008E2F90E0EBE3F4E028C0EFE1F4E0E4912B
:1025E0008E2F90E0EFE1F4E020C08330910508F0F9
:1025F000BCC0880F991FFC01E65CFE4F0190F08182
:10260000E02D89E090E014C08330910508F0ADC062
:10261000FC01EE0FFF1FEC5CFE4F0190F081E02DFE
:10262000DC01AF5CBE4F8C9190E0009709F49DC037
:102630002091E800277F2093E8002091E401309169
:10264000E5012817390708F4C90140E0009789F12E
:102650002091DC01222309F43DC02530D9F12091DD
:10266000E80023FD37C02091E80022FD2FC0209113
:10267000E80020FFEBCF4091F3002091F20030E022
:10268000342B009759F02830310540F444914093A1
:10269000F100319601972F5F3F4FF3CF41E0283093
:1026A000310509F040E02091E8002E772093E80002
:1026B000CDCF4111CDCF0AC08091DC01882351F0EC
:1026C000853041F08091E80083FD04C08091E800EE
:1026D00082FFF2CF8091E8008B778093E80045C0BD
:1026E000803809F042C08091E800877F8093E8003D
:1026F0008091DD018093F1008091E8008E77D3CE48
:10270000811133C08091E0019091E10199270297F6
:1027100064F58091E800877F8093E8001091E001E4
:102720001093DD010E944C10111106C08091E3004E
:1027300087FD02C081E001C084E08093DC0142E0BB
:1027400061EC81E00E946B1042E261EC84E00E9447
:102750006B1042E261EC82E00E946B1042E260EC9E
:1027600083E00E946B108091DC018091E80083FF80
:1027700010C08091E800877F8093E8008091EB0093
:1027800080628093EB0005C082E190E0E9EFF3E026
:102790004FCFAA96E3E00C94672B1F920F920FB6CF
:1027A0000F9211242F933F934F935F936F937F93D7
:1027B0008F939F93AF93BF93CF93DF93EF93FF9349
:1027C000C091E900CF708091EC00D82FD17080FDCE
:1027D000D0E81092E9008091F000877F8093F000AC
:1027E00078940E9402111092E9008091F0008860B4
:1027F0008093F000CD2BCF70C093E900FF91EF9153
:10280000DF91CF91BF91AF919F918F917F916F9108
:102810005F914F913F912F910F900FBE0F901F909E
:102820001895E8EDF0E080818E7F80831092E200C1
:102830001092DA001092E100A0EEB0E08C9181607D
:102840008C9380818F77808319BCA7EDB0E08C9149
:102850008E7F8C9380818F7E80831092CF0108952C
:10286000A0E0B0E0E6E3F4E10C94462BC8EDD0E044
:1028700088818F7E8883E7EDF0E0808181608083AE
:1028800084E082BF81E08093CF0188818E7F88833E
:1028900002EE10E0F80110821092DA0081EEC82EEC
:1028A000D12CF601108288818F7788838881806897
:1028B000888388818F7D888319BC1092DC011092F7
:1028C000DD011092DB011092DA0190EEE92EF12C7D
:1028D000F70180818B7F808388818160888342E0DB
:1028E00060E080E00E946B10F60180818E7F808323
:1028F000F801808181608083808188608083F70116
:1029000080818E7F8083888180618883CDB7DEB7A8
:10291000E8E00C94622B1F920F920FB60F921124D5
:102920002F933F934F935F936F937F938F939F93D7
:10293000AF93BF93EF93FF938091E10082FF09C0B3
:102940008091E20082FF05C08091E1008B7F80933F
:10295000E1008091DA0080FF2AC08091D80080FFDA
:1029600026C08091DA008E7F8093DA008091D900B2
:1029700080FF18C080E189BD82E189BD09B400FEF5
:10298000FDCF81E08093DC018091CF0181110FC0E8
:102990000E9411140E9430148091E20084608093A0
:1029A000E20005C019BC1092DC011092CF018091A9
:1029B000E10080FF17C08091E20080FF13C080918A
:1029C000E2008E7F8093E2008091E200806180933C
:1029D000E2008091D80080628093D80019BC85E025
:1029E0008093DC018091E10084FF30C08091E2009F
:1029F00084FF2CC080E189BD82E189BD09B400FE5D
:102A0000FDCF8091D8008F7D8093D8008091E10028
:102A10008F7E8093E1008091E2008F7E8093E200C0
:102A20008091E20081608093E2008091DD01882343
:102A300011F084E007C08091E30087FD02C081E0CF
:102A400001C083E08093DC018091DC018091E10092
:102A500083FF27C08091E20083FF23C08091E100C3
:102A6000877F8093E10082E08093DC011092DD019A
:102A70008091E1008E7F8093E1008091E2008E7F63
:102A80008093E2008091E20080618093E20042E066
:102A900060E080E00E946B108091F000886080937D
:102AA000F000FF91EF91BF91AF919F918F917F9136
:102AB0006F915F914F913F912F910F900FBE0F90AB
:102AC0001F9018952091E4003091E50095E6409123
:102AD000EC00842F817040FF23C08091E80080FDCE
:102AE0001DC08091DC01882399F0853099F0809198
:102AF000EB0085FD11C04091E4005091E5002417E2
:102B0000350729F3915011F09A01E1CF84E008953F
:102B100082E0089583E0089581E0089580E00895BB
:102B20004091E80042FFDDCF08950F931F93CF93AC
:102B3000DF938B01EA019091DC01943079F58F707D
:102B40008093E9008FEF9091E800815095FD06C0D9
:102B500095ED9A95F1F700008111F5CF8091E8008D
:102B600085FF1CC00E946215882361F08091E800F7
:102B70008E778093E80012C0F80181918F018093D5
:102B8000F1002197209791F38091E80085FDF4CF23
:102B90008091E8008E778093E800E4CFDF91CF91B9
:102BA0001F910F91089543E050E0BC0184E00E9422
:102BB0009515089540E250E0BC0184E00E9495150F
:102BC0000895CF93DF93EC0148E050E0BC0181E031
:102BD0000E94951588E0FE01A2EDB1E001900D92F2
:102BE0008A95E1F7DF91CF91089581E08093E0002D
:102BF00080E28093D8001092C9008FE19EE4019793
:102C0000F1F700C0000087E090EBDC018093310316
:102C100090933203A0933303B09334039CE088E194
:102C20000FB6F894A895809360000FBE9093600053
:102C3000FFCF78941F920F920FB60F9211248F93AB
:102C40009F93AF93BF938091CB019091CC01A091C2
:102C5000CD01B091CE010196A11DB11D8093CB0194
:102C60009093CC01A093CD01B093CE01BF91AF91D1
:102C70009F918F910F900FBE0F901F9018952FB7B7
:102C8000F8946091CB017091CC018091CD0190912D
:102C9000CE012FBF0895209141029091080257E084
:102CA0002917A9F030E0529FF001539FF00D112435
:102CB000E75FFD4F7181761306C07081781303C002
:102CC0007581741306C02F5F3F4F2770E9CF80E0F6
:102CD000089581E0089590912A0380914402892B00
:102CE000909143029923E1F0892B90910E01992351
:102CF00041F09091FF0297FF04C09EE122ED32E087
:102D000003C096E02AEC32E0F90120E0915028F06F
:102D100031913323D9F32F5FF9CF21111092430260
:102D200008958091410290910802891719F08F5FF0
:102D30008770FBCF0895CF93DF9380910702829530
:102D40008F7009F04EC080910602882309F449C0B3
:102D5000809141024091080250910202609101026B
:102D6000C0910302D091040277E08417D1F190E082
:102D7000789FF001799FF00D1124DF01A75FBD4F0F
:102D800014962C911497222349F111962C911197A6
:102D9000251324C02C91261321C015962C9115972C
:102DA00021111CC012962D913C9113972C1B3D0BA9
:102DB000283C310598F4809107028F7080618093E0
:102DC0000702E15FFD4F80818F708061808381E029
:102DD00092E00E94B4040E94911603C0019687708D
:102DE000C4CFDF91CF910895CF92DF92FF920F93DE
:102DF0001F93CF93DF936C010091B20180912B035D
:102E0000082BC3E0D0E010E0C8010C2E02C095955D
:102E100087950A94E2F780FD04C02197A8F7F12C6A
:102E200009C0FC2EB6018C2F0E9486240E94942497
:102E3000019799F38F2DDF91CF911F910F91FF9003
:102E4000DF90CF900895CF93DF93EC010E94F416AA
:102E5000BE010E9486240E949424DF91CF910895A0
:102E6000FC0124812223D9F0808191810E942317C3
:102E700092959F70963079F010F4925001C09A505C
:102E8000923068F4803F69F018F4883E40F409C03D
:102E9000843F29F406C0883E20F0813F11F080E095
:102EA000089581E00895A4E1B0E0E9E5F7E10C942C
:102EB000422B8C0186E0F801DE011F9601900D92F5
:102EC0008A95E1F7F8018481E58091E0892E92E00E
:102ED000992E90910502911120C0882309F463C1B5
:102EE000EE2009F442C0C8010E943017F82E882352
:102EF000E1F187E0F801D40101900D928A95E1F7A4
:102F000080910502813031F480910102909102029A
:102F10000E9423170E949B1648C1F801D080C180EF
:102F2000A280B380F0900602209103023091040247
:102F3000FF2009F4E7C0A501421B530B483C510593
:102F400008F09DC0882309F430C180910702282F22
:102F5000207F90910202222361F09C1509F460C049
:102F6000C8010E943017811163C0C8010E94B404D7
:102F70001AC19C1113C0909101029D110FC0E11064
:102F80000DC08F7080618093070281E092E00E9403
:102F9000B40480910702F801868303C1E1103AC0AE
:102FA00040E06C2D8D2D0E944B1640E06C2D8D2D38
:102FB0000E944B16E82E8111F4C0DF86C88A8F85E7
:102FC00098890E942317292F22952F70243020F4EE
:102FD0009F70223028F009C02A50223080F014C09F
:102FE000992349F0811107C013C0992321F0F801FA
:102FF0009681907F69F0805E883030F409C0803F10
:1030000038F0815F833020F0C8010E94B404EF2CB7
:10301000FE2CCBC080910702816080930702C1C063
:10302000909101029D119CCFE1109ACFF80198C0B8
:10303000EE2009F49ACF20910702822F82958F709B
:1030400090E002978CF080910102909102029987A2
:103050008887BB86AA86809105028C871D862E876D
:10306000CE0108960E94B40487E0F801A1E0B2E026
:1030700001900D928A95E1F70E949B1694C0909161
:103080000702292F207F51F481E092E00E94B404CE
:1030900087E0F40111928A95E9F783C0882309F447
:1030A00084C0809102028C110CC0809101028D11AC
:1030B00008C0E11006C0F8019683C8010E94B4045C
:1030C0006AC0C8010E943017882309F44ECFEE2051
:1030D00009F44BCF20910702822F82958F7090E0E8
:1030E000029714F280910102909102029A838983DF
:1030F000BC82AB82809105028D831E822F83CE011C
:103100000196B0CFA21AB30AF8ECAF16B10408F0DA
:1031100042C0882309F447C0FE2CEE2009F425CFD5
:10312000809102028C1129C0809101028D1125C06D
:103130009091070290FD18C0892F82958F70282FDB
:1031400030E02115310581F0F80196832F303105EB
:1031500041F08F5F982F9295907F86818F70892B99
:103160008683C8010E94B40487E0F801A1E0B2E0C0
:1031700001900D928A95E1F718C0C8010E9430179E
:10318000811172CF80910702816080930702C8018C
:103190000E94B4040AC087E0F40111928A95E9F70D
:1031A00004C0F12C02C0FF24F3948F2D6496ECE050
:1031B0000C945E2B292F953078F58E3068F590E0D1
:1031C0003EE0239F800D911D1124682F677023E03E
:1031D000969587952A95E1F7FC01EE0FFF1FE80F02
:1031E000F91FEA51FE4F40E050E080E0219130E0CD
:1031F000062E02C0369527950A94E2F721703327F0
:10320000042E01C0220F0A94EAF7822B4F5F5F4F12
:103210004330510559F7089580E00895292F9530DE
:1032200088F58E3078F590E03EE0239F800D911D6B
:103230001124282F277051E001C0550F2A95EAF775
:1032400023E0969587952A95E1F7FC01EE0FFF1F85
:10325000E80FF91FEA51FE4F20E030E070E04081B6
:10326000CB01022E02C0969587950A94E2F78170F1
:10327000819584278523842781932F5F3F4F2330B7
:10328000310569F708958093B20108959091B201D4
:1032900021E030E0F90101C0EE0F8A95EAF7D9018B
:1032A00002C0AA0FBB1F6A95E2F7BD016E2B01C0D9
:1032B000220F4A95EAF7892F8623681303C0892FC6
:1032C000822B03C02095822F89230E9443190895E1
:1032D00021E030E001C0220F8A95EAF72095809125
:1032E000B20182230E944319089590914202809571
:1032F000892380934202282F277069F4981759F088
:103300009091000392FF07C08695869586950E944E
:1033100068191092420208959091000392FB2227AF
:1033200020F9281779F080FB92F9909300036091BF
:10333000FF027091000384E090E00E94552A82E031
:103340000E947519089521E030E001C0220F8A958E
:10335000EAF78091B201822B0E944319089580936D
:103360002B03089510922A0380910E01882341F0C7
:103370008091FF0287FF04C08EE1E2EDF2E003C01E
:1033800086E0EAECF2E0DF011D928A95E9F780E041
:1033900090E00E94F71F80E090E00E94D21F109200
:1033A00044020E9449260895882321F00E94422663
:1033B0000E9449260895882339F090912A03892B89
:1033C00080932A030E9449260895882309F44DC05A
:1033D000823859F40E941C2081FF47C089E30E9473
:1033E0009B1F0E94492689E30CC0833879F40E9410
:1033F0001C2080FF3AC083E50E949B1F0E94492643
:1034000083E50E946D1F0E9449260895843859F46F
:103410000E941C2082FF29C087E40E949B1F0E94FB
:10342000492687E4EECF9CEF980F913A50F390E253
:10343000980F983050F4877091E001C0990F8A95E9
:10344000EAF7892F0E944226DECF9BE5980F933042
:1034500028F480E090E00E94F71F0895885A8B318D
:1034600020F480E090E00E94D21F0895CF9388233B
:1034700009F4D7C0C82F8238A1F40E941C2081FD16
:10348000D0C089E30E949B1F0E9449262FEF87EE40
:1034900093E0215080409040E1F700C0000089E3B4
:1034A00015C08338C1F40E941C2080FDBAC083E59A
:1034B0000E949B1F0E9449262FEF81EE94E021502D
:1034C00080409040E1F700C0000083E50E946D1F3E
:1034D0000E944926A6C08438A1F40E941C2082FDC7
:1034E000A0C087E40E949B1F0E9449262FEF81EE17
:1034F00094E0215080409040E1F700C0000087E454
:10350000E5CF8CEF8C0F813A40F58091F40288234F
:1035100019F0813051F01EC080912A03823209F0E7
:103520004CC08C2F0E94A02146C080912A03823279
:10353000C1F3C43149F018F4CB3049F03AC0C93274
:1035400019F0C83321F035C01092F40232C081E086
:10355000817031C01092F40230C080E28C0F88304C
:1035600068F4C77081E090E001C0880FCA95EAF75F
:1035700090912A03892B80932A03AACFEBE5EC0FC5
:10358000E33040F4F0E0E05CFE4F808190E00E9488
:10359000F71F47C0C85ACB3108F043C0EC2FF0E00A
:1035A000EE0FFF1FED5BFE4F808191810E94D21FC5
:1035B00038C080E0CDCF811134C080910E018823C6
:1035C000E1F08091FF0287FF18C0EC2FE695E695A9
:1035D000E695F0E0E053FD4F8281282F30E04C2F3C
:1035E000477081E090E002C0880F991F4A95E2F78A
:1035F00082239323892B61F410C0EAECF2E080ED82
:1036000092E02191C21721F08E179F07D1F705C0D4
:103610008C2F0E946D1F0E9449268C2F0E949B1F99
:1036200057CFCF9108951F93CF93DF93182FEB01BE
:103630000E94361A209741F08FE99FE00197F1F739
:1036400000C000002197F6CF812F0E94E519DF917D
:10365000CF911F9108950895A3E0B0E0E2E3FBE16C
:103660000C944A2B8C0180914F0281110AC09E015B
:103670002F5F3F4F4FEF6FEF0E941A278A81809391
:103680004F02F8018481813051F028F0823061F4DA
:1036900040914F020AC080914F0240E007C0609104
:1036A0004F0240E080E003C040E080E060E00E9424
:1036B0009B26F801848190E0019663E070E00E940F
:1036C0000C2B84832396E4E00C94662BCF93DF933A
:1036D000EC01E0ECF2E0438162818C810E94A6273C
:1036E0008C818F5F8C83DF91CF910895CF93DF938F
:1036F000EC01EC81F0E0E15CFB4F4491E0ECF2E0A6
:10370000628181810E94A6278C818F5F8C83DF91EB
:10371000CF910895A0E0B0E0E0E9FBE10C94422BEA
:103720008C0180918600909187006CE070E00E948F
:10373000F82A6017710730F0C80169E070E00E9454
:10374000F82A60C08091860090918700E090860002
:10375000F0908700E0918600F0918700C6E0D0E00D
:10376000BE010E94F82A20E030E0060F171F211D3D
:10377000311D4801590185E0880C991CAA1CBB1C0D
:103780008A95D1F7C701BE010E94F82A6F01E12C8A
:10379000F12CA7019601260F371F411D511DC501B0
:1037A000B4010E949D2A69017A01E0918600F0919E
:1037B0008700CA01B9010E94CE2A9B01AC01DF013A
:1037C0000E948A2A9B01AC01C701B6010E94CE2A41
:1037D000DC01CB012FE0B695A795979587952A95A3
:1037E000D1F7009186001091870020E030E00817A3
:1037F00019072A073B0728F460918600709187001B
:10380000CB01BC01CB01CDB7DEB7ECE00C945E2B55
:10381000682F86E090E00E94372A08958091F00298
:1038200081FF11C08D7F8093F0020E94081C80915F
:103830006F008E7F80936F008091F0028695869551
:1038400086950E94962208958091F00281FD10C015
:1038500082608093F0020E94081C1092F302109282
:10386000F2021092F10280916F00816080936F00EC
:103870000895863008F085E09091F0029770282F27
:10388000220F220F220F922B9093F002987F21E0BB
:1038900009F420E09091F00220FB90F99093F0025F
:1038A0000E94962208958091F00280FF08C08E7FCA
:1038B0008093F0020E94081C80E00E9496220895E6
:1038C0008091F00280FD13C081608093F00281300E
:1038D00019F489E08093F0028091F0020E94081CA4
:1038E0008091F0028695869586950E94962208958D
:1038F00086E090E00E94132A8093F00282FD05C0CA
:103900008DE28093F0020E94081C8091F002282F23
:1039100026952695269530E02630310524F08770CF
:1039200088628093F0028091F00280FF04C0869547
:103930008695869501C080E00E9496220895909118
:10394000C00290FF05C096959695981748F003C061
:10395000811106C090E0961718F40E94E02808959F
:1039600061E00E9485280895882311F0FA0101C0C2
:10397000FB01099508956091C0026695669570E017
:103980004BE050E08FE091E00E94AA2B892B19F4C4
:1039900081E080934C020E94381F909346028093EE
:1039A000450208958091C00280FF07C06EE070E07C
:1039B00080E592E00E940E1F0895E0E5F2E011829A
:1039C00010821282339682E0EA37F807C1F7EECF11
:1039D000A0E0B0E0EEEEFCE10C94412BFC01828013
:1039E000748081E08483EFE3F4E09490EEEBF4E004
:1039F000E4910091C3020695015810E0000F111FD9
:103A0000012F1127CAE7D2E020E5C22E22E0D22EF4
:103A1000AA24AA94B12CE919EE2EF12C22E0281543
:103A200030F08091C10288838091C2028983711035
:103A300003C01B821A824AC08B818823F9F081500F
:103A40008B832FEF829FC00111246C8170E00E9454
:103A5000F82AFB01FF27E15CFB4F8491E82FE9196D
:103A60002FEFE29FC0011124B7010E94F82A809134
:103A7000C302689FB00111247A8328C00E94032AE0
:103A8000B5010E940C2B8017910704F582E0881580
:103A900088F40E94032AB5010E940C2B88830E949F
:103AA000032A2091C2022695622F70E00E940C2BFF
:103AB000280F29831A828091C302843120F0893C27
:103AC00018F088EC01C084E18C838B8396014A81D5
:103AD000698188810E941A27259623E0C20ED11C95
:103AE00082E0C03CD80709F099CF0E94D21CCDB724
:103AF000DEB7EDE00C945D2BEF92FF920F931F93D6
:103B0000CF93DF938C01C0E5D2E0E12CF12CF801DA
:103B10008481F7E0EF16F1041CF4882339F002C029
:103B2000811104C09E014091C30202C09E0140E089
:103B30006091C2028091C1020E941A278FEFE81A99
:103B4000F80A23969EE0E916F10409F70E94D21CB8
:103B5000F801848190E00196817099278483CDB724
:103B6000DEB7E6E00C94642BA0E0B0E0EAEBFDE108
:103B70000C94422BEC014C81042F10E09801D801E9
:103B80000E94BF2A9B01AC010E948A2A6B017C0122
:103B9000E0E2F0E0E01BF10BA5E5B0E09B01AC0139
:103BA0000E948A2A4B015C019F01DF010E942D2B9C
:103BB0009B01AC010E94952A9B01AC012C0D3D1D7F
:103BC0004E1D5F1DC501B4010E949D2A822FF22E59
:103BD00099E2921728F093E0299F900111240DC0DB
:103BE00025E530E0281B3109C901880F991F280FEE
:103BF000391F37FF02C02F5F3F4F35952795122F92
:103C0000109590E5C92E92E0D92E00E085E5E82ECA
:103C1000EF1801FD02C08E2D01C08F2D9601412F9E
:103C20006091C2020E941A270F5F83E0C80ED11C68
:103C30000E3079F70E94D21C8C81811102C091E074
:103C400003C0803219F49FEF90931C0190911C01E6
:103C5000890F8C83CDB7DEB7ECE00C945E2B0F930D
:103C60001F93CF93DF93C0E5D2E0FE011182108253
:103C70001282339682E0EA37F807C1F700E010E0DD
:103C800080914E02082E000C990B0817190794F02A
:103C900080911B01082E000C990B8017910754F09E
:103CA0009E014091C3026091C2028091C1020E94B4
:103CB0001A2703C0198218821A820F5F1F4F23969A
:103CC0000E301105E9F60E94D21C80911A019091E4
:103CD0004E02980F90934E0220911B01280F2093C3
:103CE0001B01121614F49D301CF0819580931A016B
:103CF000DF91CF911F910F910895A0E0B0E0E3E82C
:103D0000FEE10C94452BFC01828180FF03C0DD2481
:103D1000DA9402C0DD24D39400E512E0C0E0D0E0E4
:103D20002EE0B22EF80111821082128294E0E92E68
:103D3000F12CC12C80914D028C0D8F302CF06B2D0D
:103D40000E94EA2A892F02C087FD825F082E000C9C
:103D5000990BC817D90791F48091C3028E9DA001D9
:103D60008F9D500D11245595479555954795980170
:103D70006091C2028091C1020E941A27CD0CF1E02D
:103D8000EF1AF108B9F621960D5F1F4FCE30D1051D
:103D900049F60E94D21C80914D0291E0D91206C0D2
:103DA000811102C08DE007C0815005C090E00196EE
:103DB000BE010E940C2B80934D02CDB7DEB7E9E027
:103DC0000C94612BEF92FF921F93CF93DF93EC0142
:103DD00080E5E82E82E0F82E10E08C81970140917A
:103DE000C3026091C202810F0E941A271E5E83E007
:103DF000E80EF11C1C3F89F70E94D21C9A818C812D
:103E000090FF02C08F5F01C081508C83DF91CF9102
:103E10001F91FF90EF900895809A089521B32E7F0F
:103E200031B331604FB7F894FC01CB01880F991F73
:103E3000680F791F6E0F7F1FE617F70789F08191D2
:103E400098E031BB000000C087FF21BB880F000055
:103E500000C000C000C021BB00C09A9591F7ECCF14
:103E60004FBF8FE594E00197F1F700C0000008957F
:103E70002FB7F8948091CB019091CC01A091CD0106
